:100000000C9474050C94BC050C94BC050C94BC05B4
:100010000C94BC050C94BC050C94BC050C94BC055C
:100020000C94BC050C94BC050C94BC050C948C136E
:100030000C943B140C94FB210C94BC050C94BC0553
:100040000C94BC050C94BC050C94BC050C946F225C
:100050000C94BC050C94BC050C94BC050C94BC051C
:100060000C94BC050C94BC050C94BC050C94BC050C
:100070000C94BC05F2111912111319121113651207
:1000800088121113DF12EE120C180C1836183618DD
:100090009118C518D31AD31ADC18D31AC719C7195F
:1000A0008D1AD31AA21AC01A041607090B0A1D1BAF
:1000B00006196405141A08151C171E1F2021232277
:1000C0002E26242D25273012182F0C13280F0D341F
:1000D0000E333136381110372B2C352A5829787BBE
:1000E00079397A504F5152726C63685680668053EA
:1000F000020103555880576D6E5462595A5B5C5D1E
:100100005E5F6F60617475663E3F403C414277447C
:1001100076466B47804365458048494A4B4C3D4D88
:100120003B4E3A7D7E7C7F730A0025303458006157
:1001300064625F686F73745F6B62645F726563763D
:100140003A20004552524F523A206D656469612051
:100150006B6579300A004552524F523A206D656402
:100160006961206B6579310A004D3A646574656395
:100170007420616761696E0A00544D353A206578D4
:10018000740A00556E6B6E6F776E0A00544D353AE7
:100190002064656661756C740A005D206370693D5A
:1001A00025640A002530325820004578743A205BD7
:1001B00000436C6173736963203230306370690A85
:1001C00000436C6173736963203130306370690A76
:1001D000004D3A61646472256420726567333A2089
:1001E000253034580A004D3A6D6F76652066616996
:1001F0006C0A004D3A61646472256420726567334D
:100200003A20253034580A004D3A5B423A253032C4
:100210005820583A25642825642920593A2564280D
:1002200025642920413A25645D0A004D3A5B25305A
:10023000325820253032582025303258202530328F
:100240005820253032585D0A0020616464723A25D6
:10025000642C20726567333A253034580A000A53FB
:1002600063616E3A0A004D65646961206B6579735C
:100270000A0068616E646C65723A20253032582C31
:100280002049534F3A2025730A000A4B6579626F63
:100290006172643A0A007300530052000A4B657998
:1002A000626F6172642073746172742E0A000A5561
:1002B000534220636F6E666967757265642E0A002B
:1002C0000A0A544D4B3A63653565353635662F4C11
:1002D0005546410A0A002E03410044004200200016
:1002E0006B006500790062006F00610072006400BD
:1002F000200063006F006E007600650072007400DD
:100300006500720000000E0374002E006D002E00C8
:100310006B002E00000004030904090274000401AC
:1003200000A03209040000010301010009211101AC
:1003300000012240000705810308000A09040100AA
:100340000103010200092111010001224D000705EE
:10035000820308000A0904020001030000000921C9
:10036000110100012236000705830308000A090471
:1003700003000203000000092111010001222200F4
:100380000705840320000107050403200001120172
:10039000100100000008EDFEDB0A0101010200016E
:1003A0000631FF0974A1010975150026FF0095208B
:1003B000750881020976150026FF009520750891C1
:1003C00002C005010980A10185021601002637003F
:1003D0001A81002AB700751095018100C0050C092B
:1003E00001A1018503160100269C021A01002A9C26
:1003F00002751095018100C005010902A1010901E2
:10040000A1000509190129051500250195057501AA
:1004100081029501750381010501093009311581BA
:10042000257F95027508810609381581257F95017C
:1004300075088106050C0A38021581257F9501751E
:10044000088106C0C005010906A101050719E029B8
:10045000E715002501950875018102950175088150
:100460000105081901290595057501910295017588
:100470000391010507190029FF150026FF009506C5
:1004800075088100C0636F6E73756D65723A2025C3
:100490003034580A0073797374656D3A202530340E
:1004A000580A000A002530325820006B6579626FC7
:1004B0006172643A20004C45443A20253032580A93
:1004C00000253032583A202530386225730A0072F0
:1004D0002F632030313233343536370A00290A0091
:1004E0002575002F002575005D280025640020007B
:1004F000256400200025640020002564007C002580
:10050000303258006D6F7573656B6579205B62746E
:100510006E7C782079207620685D287265702F6166
:10052000636C293A205B006D6B5F776865656C5F73
:1005300074696D655F746F5F6D6178203D2025641F
:100540000A006D6B5F776865656C5F6D61785F73DE
:1005500070656564203D2025640A006D6B5F7469D9
:100560006D655F746F5F6D6178203D2025640A00C2
:100570006D6B5F6D61785F7370656564203D2025EC
:10058000640A006D6B5F696E74657276616C203D04
:100590002025640A006D6B5F64656C6179203D20E5
:1005A00025640A006D6B5F776865656C5F74696DC3
:1005B000655F746F5F6D6178203D2025640A006D72
:1005C0006B5F776865656C5F6D61785F737065659B
:1005D00064203D2025640A006D6B5F74696D655F62
:1005E000746F5F6D6178203D2025640A006D6B5F3C
:1005F0006D61785F7370656564203D2025640A0035
:100600006D6B5F696E74657276616C203D20256448
:100610000A006D6B5F64656C6179203D2025640A7A
:10062000000A00257500363A20776865656C5F74AE
:10063000696D655F746F5F6D61783A20000A00250F
:100640007500353A20776865656C5F6D61785F731A
:10065000706565643A20000A00257500343A2074FC
:10066000696D655F746F5F6D61783A20000A0025DF
:100670007500333A206D61785F73706565643A2068
:10068000000A00257500323A20696E746572766141
:100690006C286D73293A20000A00257500313A2034
:1006A00064656C6179282A31306D73293A20000A1B
:1006B000092D2056616C756573202D0A004D3E0092
:1006C0004D25643E20003F007365742064656661BB
:1006D000756C740A00433E2000776865726520647B
:1006E000656C74613A20637572736F723D25642C7A
:1006F00020776865656C3D25640A536565206874DC
:1007000074703A2F2F656E2E77696B697065646916
:10071000612E6F72672F77696B692F4D6F757365E7
:100720005F6B6579730A000A092D204D6F7573653B
:100730006B6579202D0A4553432F713A097175690C
:10074000740A313A0964656C6179282A31306D7315
:10075000290A323A09696E74657276616C286D7384
:10076000290A333A096D61785F73706565640A34EC
:100770003A0974696D655F746F5F6D61780A353A27
:1007800009776865656C5F6D61785F737065656436
:100790000A363A09776865656C5F74696D655F74E0
:1007A0006F5F6D61780A0A703A097072696E742021
:1007B00076616C7565730A643A09736574206465C3
:1007C0006661756C74730A75703A092B310A646F2F
:1007D000776E3A092D310A706775703A092B3130FE
:1007E0000A7067646F776E3A092D31300A0A7370A8
:1007F000656564203D2064656C7461202A206D610C
:10080000785F7370656564202A2028726570656161
:1008100074202F2074696D655F746F5F6D61782936
:100820000A003F004D3E2000433E20004C25640A54
:10083000000A092D20436F6E736F6C65202D0A45E9
:1008400053432F713A09717569740A6D3A096D6FD6
:100850007573656B65790A000A092D204D6167691A
:1008600063202D0A643A0964656275670A783A095B
:100870006465627567206D61747269780A6B3A0904
:100880006465627567206B6579626F6172640A6D79
:100890003A096465627567206D6F7573650A763A0B
:1008A0000976657273696F6E0A733A0973746174BD
:1008B00075730A633A09636F6E736F6C65206D6FB1
:1008C00064650A302D343A096C61796572302D34D3
:1008D000284631302D4634290A506175733A096231
:1008E0006F6F746C6F616465720A003F0074696DAC
:1008F00065725F72656164333228293A202530348D
:100900006C580A006B6579626F6172645F69646C30
:10091000653A2025580A006B6579626F6172645FE1
:1009200070726F746F636F6C3A2025580A00686F9D
:1009300073745F6B6579626F6172645F6C65647319
:1009400028293A2025580A000A092D205374617479
:100950007573202D0A004743433A20352E342E303C
:10096000204156522D4C4942433A20322E302E30EF
:10097000204156525F415243483A206176723335E6
:100980000A004F5054494F4E533A204C554641208F
:100990004D4F5553454B45592045585452414B45B1
:1009A0005920434F4E534F4C4520434F4D4D414EE0
:1009B00044204B45594D41505F53454354494F4E98
:1009C00020343039360A004255494C443A20636598
:1009D000356535363566202830383A34393A353081
:1009E000204665622031332032303230290A0056E9
:1009F00049443A2030784645454428742E6D2E6B84
:100A00002E29205049443A20307830414442284130
:100A10004442206B6579626F61726420636F6E7609
:100A2000657274657229205645523A20307830310B
:100A300030310A00444553433A20636F6E76657245
:100A40007420414442206B6579626F617264207446
:100A50006F205553420A000A092D205665727369AA
:100A60006F6E202D0A000A6D6F7573653A206F66F0
:100A7000660A000A6D6F7573653A206F6E0A000A88
:100A80006B6579626F6172643A206F66660A000A6C
:100A90006B6579626F6172643A206F6E0A000A6D4D
:100AA00061747269783A206F66660A000A6D617433
:100AB0007269783A206F6E0A000A64656275673A57
:100AC000206F6E0A000A64656275673A206F666679
:100AD0000A000A0A626F6F746C6F616465722E2E71
:100AE0002E2000433E20000011241FBECFEFD4E093
:100AF000DEBFCDBF04B603FE28C080918003909175
:100B00008103A0918203B09183038730904BA7406B
:100B1000B04BD9F41092800310928103109282039B
:100B20001092830314BE0FB6F894A89580916000CC
:100B3000886180936000109260000FBE10920108DF
:100B400010920008E0E0F8E3099511E0A0E0B1E0C0
:100B5000ECEDF5E502C005900D92A235B107D9F78D
:100B600023E0A2E5B1E001C01D92A038B207E1F791
:100B70000E94150F0C94EC2A0C940000FF93EF9345
:100B8000E0915201F0915301309709F00995EF91EE
:100B9000FF910895FC018591803011F0EFDFFBCFCC
:100BA0000895FF27E0E230E247FF0CC0419597FF30
:100BB00009C0EDE26095709580959095611D711D5D
:100BC000811D911D27FF02C0219530E350E2AA2725
:100BD000660F771F881F991FAA1FA41710F0A41B68
:100BE00063955A95A9F7AA3008F0A95FA05DAF9365
:100BF000F395611571058105910541F7ED3211F409
:100C0000EF93F395F21718F43F93F395FBCF8F9181
:100C1000B5DFFA95E1F70895E991F9918591803072
:100C200021F0853219F0AADFF9CF089520E0E89489
:100C300055915532C1F3503311F4689455915A339C
:100C400048F4505390F3220F022E220F220F200D52
:100C5000250FF4CF0EF4219589919991533619F30C
:100C6000533729F1533559F1BC0188279927E89466
:100C70005C3621F48991999168945591543639F4F0
:100C800046EF7EF077FF0DC08FEF9FEF0AC055371C
:100C90004AE039F0583540E121F0523642E009F09F
:100CA0000895FF93EF937DDFEF91FF91B7CFFF930F
:100CB000EF93FC0181918030B9F360DFFBCFFF93AC
:100CC000EF9368DFF1CFDF93CF93CDB7DEB72596F3
:100CD000A3DFCF91DF910895282F2770E82FE695A5
:100CE000E695E695EF70F0E0E05AFE4F87FF0AC008
:100CF00081E090E001C0880F2A95EAF78095908105
:100D0000892308C081E090E001C0880F2A95EAF7A6
:100D10009081892B808308950F931F93CF93DF9346
:100D20008EE592E09F938F930E9463060F900F9041
:100D3000C0E0D0E009E412E063E08C2F0E94D90B00
:100D4000009771F09F938F93DF93CF931F930F932F
:100D50000E9463060F900F900F900F900F900F90CE
:100D60002196C031D10541F7DF91CF911F910F91AD
:100D700008953F924F925F926F927F928F929F92CF
:100D8000AF92BF92CF92DF92EF92FF920F931F9399
:100D9000CF93DF93CDB7DEB728970FB6F894DEBFB9
:100DA0000FBECDBF8091590190915A010E944522FA
:100DB0000C9708F487C20E942D2290935A018093C9
:100DC000590180915701909158010E944522893E16
:100DD000934008F458C10E942D22909358018093AB
:100DE000570153E8452E51E0552E6CE8662E61E020
:100DF000762E7AEAC72E71E0D72EE4EAAE2EE1E035
:100E0000BE2E63E083E00E94D90B8C01009709F4A9
:100E10003AC11F938F931F9283E08F9383EF91E0EA
:100E20009F938F930E94630683E00E94480C412F9A
:100E30004F602EEF63E083E00E94360C8FE00E944B
:100E4000480C63E08FE00E94D90B8C010F900F904B
:100E50000F900F900F900F90009729F0982E44E676
:100E6000E42EF12C69C086EE91E09F938F930E944F
:100E700063060F900F90C5CF8FE00E94480C24E0CE
:100E8000412F63E08FE00E94360C63E08FE00E9408
:100E9000D90B8C01982E31E083130FC08FE00E9494
:100EA000480C22E0412F63E08FE00E94360C63E0A3
:100EB0008FE00E94D90B8C01982E1F930F931F92E5
:100EC0008FE08F9381ED91E09F938F930E94630653
:100ED0000F900F900F900F900F900F9031E09312A2
:100EE00030C081EC91E09F938F930E946306F09253
:100EF0001301E09212010F900F908FE00E94480CB6
:100F0000412F407F4A602EEF63E08FE00E94360C55
:100F10008AE00E94480C63E08FE00E94D90B8C01AC
:100F2000982E892B09F46DCF89E691E09F938F93DA
:100F30000E9463060F900F908FEF890D823088F426
:100F40009BCF32E093120DC081EB91E09F938F9382
:100F50000E94630688EC90E0909313018093120145
:100F6000CACF94E0991271C028E0AE014F5F5F4F85
:100F700061E08FE00E94560B863050F02D813E815B
:100F8000322723273227309313012093120106C002
:100F9000F0921301E09212018823B9F1882E912C6E
:100FA0001F928F93DF92CF920E9463060F900F9053
:100FB0000F900F90312C832D032C000C990B88156A
:100FC00099059CF4E1E0F0E0EC0FFD1FE80FF91F3C
:100FD00080811F928F93BF92AF920E9463063394D9
:100FE0000F900F900F900F90E6CF809113018F9389
:100FF000809112018F932AE931E03F932F930E9451
:1010000063060F900F900F900F9089818B34C1F47D
:101010008A818D34A9F48B818C3491F48C81813355
:1010200079F47F926F920E9463068FE00E94480CD1
:101030002EEF412F407F63E08FE00E94360C5BCFA4
:101040005F924F920E94630656CF82E3981255CF6B
:1010500029E731E03F932F930E9463068FE00E94BF
:10106000480C28E04AE051E062E08FE00E94FF0B6C
:101070008FE00E94480C28E042E051E062E08FE0FF
:101080000E94FF0B38CF25E0AE014F5F5F4F60E05D
:101090008AE00E94560B182F823010F481E010C1B4
:1010A0008D811F928F938C811F928F938B811F92C2
:1010B0008F938A811F928F9389811F928F938BE2E6
:1010C00092E09F938F930E9463060FB6F894DEBF61
:1010D0000FBECDBF123049F4998196FB992790F944
:1010E0008A8186FB882780F90AC0FE01E10FF11D85
:1010F000808186FB992790F982FB882780F948EF49
:1011000058E81530E0F4212F012E000C330BE1E0FC
:10111000F0E0EC0FFD1FE20FF31F911102C05083AE
:1011200001C04083882349F0E1E0F0E0EC0FFD1FAF
:10113000E20FF31F2081276020831F5FE2CFED8144
:10114000E3FF02C020E001C020E8E7FF20643C810B
:1011500033FF206237FF20614B8143FF286047FF48
:1011600024605A8157FF2260698167FF21602093C4
:101170005B01A42FA077B0E083E0AA0FBB1F8A9584
:10118000E1F7932F9077892F90E076E0880F991FF1
:101190007A95E1F7A82BB92B6F77CD01862BAE2F6F
:1011A000A077B0E0BA2FAA27BB0FA82BB92B5F7787
:1011B000F0E0FE2FEE27F295FF0FF07EE52B477053
:1011C00050E05695542F442757954795CF01842BCF
:1011D000952B3770E32FF0E0FE2FEE27FF0FFF0F68
:1011E000E82BF92B40915601042F042E000C110B13
:1011F000CF01B8010E94AD2A81383FEF930714F464
:1012000081E89FEF91958195910981385FEF95076E
:1012100014F481E89FEF382F319530935C01CD01B4
:10122000B8010E94AD2A81385FEF950714F481E878
:101230009FEF91958195910981385FEF950714F49F
:1012400081E89FEF819580935D011F934F93BF933A
:10125000AF93482F082E000C550B5F938F93FF938D
:10126000EF93832F032E000C990B9F933F931F92B4
:101270002F9388E092E09F938F930E9463068BE503
:1012800091E00E94D91480915601482F082E000C3D
:10129000550B0FB6F894DEBF0FBECDBF20911201E3
:1012A00030911301283C310518F428E030E002C0E9
:1012B00024E030E091E0421753070CF090E0890FF2
:1012C0008093560128960FB6F894DEBF0FBECDBFAF
:1012D000DF91CF911F910F91FF90EF90DF90CF9012
:1012E000BF90AF909F908F907F906F905F904F9046
:1012F0003F9008951F93CF93DF93C0910001D09149
:1013000001018FEF9FEF9093010180930001CF3F88
:101310008FEFD80709F074C0809154019091550166
:101320000E9445220C9710F480E0BAC00E942D2242
:10133000909355018093540182E00E94FC0BEC01D4
:10134000892B09F05DC080917101882309F458C090
:1013500087E00E94FC0B009709F452C09C012F7794
:10136000332722303105A1F048F42115310569F009
:101370002130310599F480788A641AC02330310510
:1013800051F02F373105A1F009C08078826410C078
:10139000807889640DC0807888640AC086E591E011
:1013A0009F938F930E9463060F900F9081E178C006
:1013B000292F33272F7733272130310579F050F04B
:1013C0002230310579F02330310581F49078EC0139
:1013D000D86416C09078EC01D26412C09078EC0109
:1013E000DA640EC09078EC01D9640AC083E491E01D
:1013F0009F938F930E9463060F900F9080E150C0DF
:101400008091620381FF18C0209709F48DCF8FE28D
:1014100091E00E94CA05DF93CF938AE291E09F9307
:101420008F930E94630688E291E00E94CA050F90A4
:101430000F900F900F9003C0209709F475CFCF370E
:101440008FE7D80711F48FE705C0CF3F8FEFD8079C
:1014500021F48FEF0E946C0622C08D2F1C2FDF3FDE
:1014600011F48C2F1FEF90917001992359F0982F50
:101470009F77923319F480788A6004C09A3011F40F
:10148000807882630E946C061F3F49F0812F90E0B4
:10149000982F88278F6F909301018093000181E03E
:1014A000DF91CF911F910895E82FF0E0E05AFE4FB1
:1014B00080810895682F609582E00C945E0C809185
:1014C0006203816080936203569A5E9A0E94520B77
:1014D0002FEF83ED90E3215080409040E1F700C072
:1014E00000000E948C068AE892E09F938F930E94EE
:1014F000630663E082E00E94D90B99270F900F905A
:101500008131910539F190F48730910519F138F462
:101510009C01245031092230310500F51BC089306F
:101520009105C1F08D309105C9F414C08D3191053C
:1015300089F038F48431910569F08931910571F4AD
:1015400009C0843C910531F0873C910519F0813C3C
:10155000910521F421E02093700102C010927001E6
:1015600020917001211103C021E331E002C02DE27E
:1015700031E03F932F939F938F9382E792E09F9365
:101580008F930E94630663E087E00E94D90B99273E
:1015900021E00F900F900F900F900F900F908230DE
:1015A000910509F020E020937101029741F486E64D
:1015B00092E09F938F930E9463060F900F9023E019
:1015C00042E063E082E00E94360CE0E6F1E0119236
:1015D00021E0E037F207D9F70E9484140E945A0AEA
:1015E0000E948C06569A5E980895509A83E091E086
:1015F0000197F1F700C0000050989AEB9A95F1F727
:1016000000C00895509A8AEB8A95F1F700C050986F
:1016100083E091E00197F1F700C000000895EF9298
:10162000FF920F931F93CF93DF93C0E0D0E090E839
:10163000E92EF12C082F10E0C7010C2E02C0959561
:1016400087950A94E2F780239123892B19F00E9451
:10165000020B02C00E94F50A2196C830D10561F73D
:10166000DF91CF911F910F91FF90EF900895509AC5
:1016700083EF9BE00197F1F700C000000C94020B90
:10168000489B06C023E02A95F1F700000197C1F7B7
:101690000895489906C023E02A95F1F700000197C4
:1016A000C1F708955898509808950895EF92FF92C1
:1016B0000F931F93CF93DF93182FC62F7A01D22F4A
:1016C00080E0422F50E0282F082E000C330B241707
:1016D000350734F4F701E20FF31F10828F5FF3CF69
:1016E000F8940E94370B812F8295807FCC608C2BE1
:1016F0000E940F0B0E94F50A84EF91E00E94490BB3
:10170000892B19F48AE992E01AC084EF91E00E94D3
:10171000400B892B19F4789480E044C088E290E073
:101720000E94490B892B19F488E992E008C084E6ED
:1017300090E00E94400B892B51F486E992E09F9340
:101740008F930E94630678940F900F90E5CFC0E0CE
:1017500082E890E00E94490B8823F9F08C01112760
:10176000C8010E94400B8823C1F09C2F9695969546
:1017700096959D1780F4F701E90FF11D9081990F5F
:1017800022E830E0201B310B081B1109201731071C
:101790000CF491609083CF5FD9F678948C2F869566
:1017A00086958695DF91CF911F910F91FF90EF90D5
:1017B0000895CF93DF93CDB7DEB728970FB6F8948F
:1017C000DEBF0FBECDBF28E0AE014F5F5F4F0E946E
:1017D000560B823031F489819A819827892798277E
:1017E00002C080E090E028960FB6F894DEBF0FBEEE
:1017F000CDBFDF91CF91089560E00C94D90BEF92AB
:10180000FF921F93CF93DF93182FD62F7A01C22F09
:10181000F8940E94370B812F8295807FD8608D2BA2
:101820000E940F0B0E94F50A8FE193E00197F1F7F8
:1018300000C000000E94020B10E0D0E0812F012EBA
:10184000000C990B8C179D0744F4F701E80FF91F62
:1018500080810E940F0B1F5FF1CF0E94F50A7894E0
:10186000DF91CF911F91FF90EF900895CF93DF9379
:1018700000D0CDB7DEB749832A8322E0AE014F5FA7
:101880005F4F0E94FF0B0F900F90DF91CF91089553
:10189000CF93C82FF8940E94370B8C2F8295807FAE
:1018A00081600E940F0B0E94F50A8FE193E001977F
:1018B000F1F700C000007894CF910895262F27708B
:1018C00040E062E00C94360C80917E020895CF9344
:1018D000DF9300D01F92CDB7DEB79C0180917703D4
:1018E000843019F593E099833B832A839093E90030
:1018F0008FEF9091E800815095FD06C095ED9A9587
:10190000F1F700008111F5CF8091E80085FF0DC04F
:1019100040E050E063E070E0CE0101960E94C51007
:101920008091E8008E778093E8000F900F900F90E1
:10193000DF91CF910895CF93DF9300D01F92CDB761
:10194000DEB720917703243031F522E029838058D7
:1019500091099B838A8383E08093E9008FEF9091C4
:10196000E800815095FD06C095ED9A95F1F70000CD
:101970008111F5CF8091E80085FF0DC040E050E077
:1019800063E070E0CE0101960E94C5108091E800EE
:101990008E778093E8000F900F900F90DF91CF919A
:1019A0000895209177032430F1F422E02093E90098
:1019B0002FEF3091E800215035FD06C035ED3A9506
:1019C000F1F700002111F5CF2091E80025FF0BC0B1
:1019D00040E050E065E070E00E94C5108091E800B2
:1019E0008E778093E8000895CF93DF93209177035B
:1019F000243049F521E02093E90021E8215059F0F5
:101A00003091E80035FD07C0EFE3F1E03197F1F7E1
:101A100000C00000F3CF2091E80025FF14C0EC01C6
:101A200040E050E068E070E00E94C5108091E8005E
:101A30008E778093E80088E0FE01A6E7B2E001908F
:101A40000D928A95E1F7DF91CF910895CF93C091E0
:101A50007401C1110BC00E943922643C7940810598
:101A6000910520F081E080937401C1E08C2FCF912B
:101A70000895FF920F931F93CF93DF93D82F0FB644
:101A800007FE83C080917703843081F08091170135
:101A900090E001962091190130E082239323209158
:101AA000180130E08217930709F0C9C00E94260D83
:101AB000811110C08091170190E0019620911901C9
:101AC00030E0822393232091180130E0821793079E
:101AD00009F0B5C00E942D228C01C091E900CF70A1
:101AE0009091EC00892F817090FD80E8C82B84E0F4
:101AF0008093E90085E0F82E8091EB0085FD42C0DF
:101B00008091EB0080FF3EC08091EE0087FF3AC0DD
:101B10008091180190911701981709F457C090917E
:101B2000E80095FF8AC0E0911501F0911601E80FD9
:101B3000F11D20818F5F90911901892380931801F5
:101B40002093F1008091E80085FDE2CF8091E800CC
:101B500080FFDECF8091E8008E778093E800F092DE
:101B60001401D6CF8091170190E0019620911901C0
:101B700030E0822393232091180130E082179307ED
:101B800009F448C0CF70C093E90040911701842F39
:101B900090E001962091190130E082239323209157
:101BA000180130E08217930709F44CC0E091150149
:101BB000F0911601E40FF11DD083809117018F5F22
:101BC000909119018923809317013CC08091E8000E
:101BD00085FF33C0D093F10081E09091F20099230A
:101BE00091F09091E80090FF0EC09091E80095FF71
:101BF00003C01092F100F9CF9091E8009E77909386
:101C0000E800F0921401882309F4ACCFCF70C093A0
:101C1000E90018C080911401882309F4B3CF0E9411
:101C20002D229C018017910711F4890165CF9091B5
:101C30001401915090931401F8CF80E0CECF4091E1
:101C40001701B4CF80E0DF91CF911F910F91FF90EA
:101C500008950895089542E061EC81E00E943E10ED
:101C600042E061EC82E00E943E1042E061EC83E0E1
:101C70000E943E1042E261EC84E00C943E108091A0
:101C80007903833009F453C030F4813071F082302D
:101C900009F48CC008958A3009F478C08B3009F4B7
:101CA0005EC0893009F09AC020C080917803813AE3
:101CB00009F094C08091E800877F8093E8008091CC
:101CC0007C0390917D03892B21F468E086E792E004
:101CD00003C060E080E090E070E00E94101180910D
:101CE000E8008B778093E800089580917803813233
:101CF00009F074C080917C0390917D03892B09F0D9
:101D00006DC08091E800877F8093E8008091E800B3
:101D100082FD05C0809177038111F8CF5FC080916B
:101D2000F10080937E028091E8008B7753C0809110
:101D30007803813A09F052C080917C0390917D0331
:101D4000892B09F04BC08091E800877F8093E800E1
:101D50008091E80080FFFCCF8091240136C0809103
:101D600078038132D9F580917C0390917D03892B92
:101D7000A9F58091E800877F8093E8000E947310A6
:101D800080917A03809324010C94BC17809178038E
:101D9000813221F58091E800877F8093E8000E94DE
:101DA000731080917B0380937F0208958091780364
:101DB000813AA1F48091E800877F8093E8008091C8
:101DC000E80080FFFCCF80917F028093F10080913A
:101DD000E8008E778093E8000C947310089580914A
:101DE0007E028093750110927E020E94ED150C9484
:101DF000BC170C94EF0E0E94BA21809175038823C2
:101E000029F00E94E32181110C94281008950E946A
:101E1000F7218091750180937E0208950C94070F3D
:101E200008950C94100F0C94100FCF9384B7877FF4
:101E300084BF0FB6F894A895809160008861809364
:101E40006000109260000FBE90E080E80FB6F8943A
:101E500080936100909361000FBE89E39DE00E9432
:101E60008D218AE191E00E947F1480EC92E00E9433
:101E7000CA050E94130F0E943E150E9429130E945A
:101E80007C138091E20084608093E20078940E9449
:101E9000401580917703843019F00E94100FF9CF1C
:101EA0008EEA92E00E94CA050E94110F8CE992E02E
:101EB0000E94CA05C4E080917703853019F40E941E
:101EC000FB0EF9CF0E9446152091E4003091E50009
:101ED00080917201909173012817390761F3809105
:101EE000E4009091E50090937301809372010E9449
:101EF000260D882301F3809177038430E1F68091E9
:101F0000E9008F702091EC00922F917020FD90E8F5
:101F1000892BC093E9009091EB0090FF3FC0909116
:101F2000EE0097FF3BC090911801209117012917EF
:101F300009F12091E80025FF1DC0E0911501F09105
:101F40001601E90FF11D30819F5F20911901922345
:101F5000909318013093F1009091E80095FDE3CF44
:101F60009091E80090FFDFCF9091E8009E779093EA
:101F7000E800D9CF9091F200992381F09091E80088
:101F800090FF0CC09091E80095FF03C01092F10003
:101F9000F9CF9091E8009E779093E8008F7080933E
:101FA000E90089CF292F332723303105C9F060F4A8
:101FB0002130310581F02230310509F041C084E73C
:101FC00090E02AE133E040C021323105E1F02232D5
:101FD000310531F135C082E190E02EE833E034C0C4
:101FE00099278130910549F028F0029749F5E6EDEF
:101FF000F2E005C0E6E1F3E002C0E6E0F3E0849140
:1020000090E09F0121C064307105D0F4660F771F06
:10201000FB01E05CFE4F2081318189E090E014C03B
:102020006430710568F4FB01EE0FFF1FE85CFE4FA2
:1020300020813181FB01EC5CFE4F808190E004C087
:1020400080E090E020E030E0FA01318320830895C1
:1020500084E089BD86E089BD09B400FEFDCF809192
:10206000D8008F7D8093D8008091E00082608093BB
:10207000E0008091E00081FDFCCF0895982F95301D
:1020800068F59093E900981739F07091EC00209171
:10209000ED005091F00003C0242F762F50E021FD79
:1020A00002C09F5FECCF3091EB003E7F3093EB009E
:1020B0003091ED003D7F3093ED003091EB003160C9
:1020C0003093EB007093EC002093ED005093F00000
:1020D0002091EE0027FDE5CF80E008958F7080937A
:1020E000E90081E008958091780387FF11C0809115
:1020F000E80082FD05C0809177038111F8CF11C0FF
:102100008091E8008B770BC080917703882349F09A
:102110008091E80080FFF8CF8091E8008E7780936F
:10212000E80008952091E4003091E50095E64091A3
:10213000EC00842F817040FF23C08091E80080FD77
:102140001DC080917703882399F0853099F08091A4
:10215000EB0085FD11C04091E4005091E50024178B
:10216000350729F3915011F09A01E1CF84E00895E9
:1021700082E0089583E0089581E0089580E0089565
:102180004091E80042FFDDCF0895CF92DF92EF92B9
:10219000FF920F931F93CF93DF93EC018B017A0192
:1021A0000E949210811133C0E114F10439F0F7015B
:1021B00080819181081B190BC80FD91FC12CD12C0C
:1021C0000115110519F18091E80085FD16C0809177
:1021D000E8008E778093E800E114F10449F0F701FC
:1021E00080819181C80ED91ED182C08285E00FC046
:1021F0000E949210882321F30AC089918093F100F4
:1022000001501109FFEFCF1ADF0ADACF80E0DF912A
:10221000CF911F910F91FF90EF90DF90CF90089595
:1022200020917E0330917F032617370748F0611510
:10223000710539F42091E8002E772093E80001C061
:10224000B901FC0120E06115710561F1809177030E
:102250008823D9F18530D9F18091E80083FD39C018
:102260008091E80082FD2BC08091E80080FFEBCFD9
:102270008091F20090E06115710551F08830910570
:1022800038F421912093F100615071090196F3CF48
:1022900021E0089709F020E08091E8008E77809394
:1022A000E800D1CF2111D2CF0AC0809177038823D3
:1022B00061F0853061F08091E80083FD0AC0809173
:1022C000E80082FFF2CF80E0089582E0089583E085
:1022D000089581E0089520917E0330917F032617B1
:1022E000370748F06115710539F42091E8002E7721
:1022F0002093E80001C0B901FC0120E061157105DF
:1023000079F180917703882309F43DC0853009F481
:102310003CC08091E80083FD3AC08091E80082FDD6
:102320002CC08091E80080FFE9CF8091F20090E01E
:102330006115710559F08830910540F4249120937E
:10234000F1003196615071090196F2CF21E00897B2
:1023500009F020E08091E8008E778093E800CECFEE
:102360002111CFCF0AC080917703882361F0853097
:1023700061F08091E80083FD0AC08091E80082FF4F
:10238000F2CF80E0089582E0089583E0089581E02F
:1023900008951F93CF93DF93CDB7DEB7AA970FB6FB
:1023A000F894DEBF0FBECDBFE8E7F3E08091F10007
:1023B000819323E0E038F207C9F70E943F0E809135
:1023C000E80083FF2EC18091780390917903492F13
:1023D00050E04A30510508F024C1FA01E65CFF4F95
:1023E0000C94D22A803821F0823809F01AC108C032
:1023F0008091740390917503992389F082600FC0D6
:1024000080917C038F70853008F00BC18093E900C8
:102410008091EB0085FB882780F91092E90090916C
:10242000E800977F9093E8008093F1001092F1000C
:10243000D1C0282F2D7F09F0F4C0882319F08230F5
:1024400061F0EFC080917A03813009F0EAC09330E7
:1024500009F080E0809375032EC080917A0381118A
:102460002AC080917C038F702FEF280F243008F052
:10247000D8C08093E9002091EB0020FF1CC093306E
:1024800021F48091EB00806214C09091EB00906188
:102490009093EB0021E030E0A90102C0440F551FEA
:1024A0008A95E2F74093EA001092EA008091EB00EF
:1024B00088608093EB001092E9008091E800877FAC
:1024C0008093E8000E947310ACC08111AAC01091E3
:1024D0007A031F778091E3008078812B8093E3005B
:1024E0008091E800877F8093E8000E9473108091BC
:1024F000E80080FFFCCF8091E30080688093E300D8
:10250000111102C082E001C083E08093770389C08B
:102510008058823008F085C080917A0390917B03C7
:102520008C3D53E0950779F583E08A838AE28983BD
:102530004FB7F894DE01139620E03EE051E2E32F1E
:10254000F0E050935700E49120FF03C0E295EF7054
:102550003F5FEF708E2F90E0EA3010F0C79601C019
:10256000C0968D939D932F5F243149F74FBF809183
:10257000E800877F8093E8006AE270E0CE01019670
:102580000E94101116C060917C0370917D03AE0112
:102590004F5F5F4F0E94D20FBC01892B09F441C0ED
:1025A0009091E800977F9093E80089819A810E943A
:1025B0006B118091E8008B778093E80032C08038FF
:1025C00081F58091E800877F8093E8008091730314
:1025D0008093F1008091E8008E7772CF811121C045
:1025E00080917A0390917B0399270297D4F480918C
:1025F000E800877F8093E80080917A0380937303DB
:102600000E94731080917303811106C08091E300D2
:1026100087FD02C081E001C084E0809377030E94BF
:102620002B0E8091E80083FF0AC08091E800877F2D
:102630008093E8008091EB0080628093EB00AA9683
:102640000FB6F894DEBF0FBECDBFDF91CF911F91C3
:1026500008950E9486130E948913E0EEF0E08081C5
:1026600081608083E8EDF0E080818F77808319BC02
:10267000E3E6F0E080818160808310927603089524
:102680000E9486130E9489138091D8008F778093CF
:10269000D8008091D80080688093D8008091D800BD
:1026A0008F7D8093D80084E089BD86E089BD09B420
:1026B00000FEFDCF10927703109273031092750302
:1026C0001092740342E060E080E00E943E1080912E
:1026D000E1008E7F8093E1008091E2008160809331
:1026E000E2008091E20088608093E2008091E00047
:1026F0008E7F8093E0000895E3E6F0E080818E7F96
:10270000808381E0809376030C9440131092E20062
:1027100008951092E10008951F920F920FB60F9244
:1027200011242F933F934F935F936F937F938F93D6
:102730009F93AF93BF93EF93FF938091E10082FF4C
:102740000BC08091E20082FF07C08091E1008B7F87
:102750008093E1000E942A0E8091E10080FF19C061
:102760008091E20080FF15C08091E2008E7F80930F
:10277000E2008091E20080618093E2008091D800C5
:1027800080628093D80019BC85E0809377030E9413
:10279000F90E8091E10084FF30C08091E20084FF57
:1027A0002CC084E089BD86E089BD09B400FEFDCF60
:1027B0008091D8008F7D8093D8008091E1008F7E3A
:1027C0008093E1008091E2008F7E8093E20080910F
:1027D000E20081608093E20080917303882311F00E
:1027E00084E007C08091E30087FD02C081E001C062
:1027F00083E0809377030E940E0F8091E10083FFB6
:1028000029C08091E20083FF25C08091E100877F8D
:102810008093E10082E080937703109273038091AC
:10282000E1008E7F8093E1008091E2008E7F8093B3
:10283000E2008091E20080618093E20042E060E08B
:1028400080E00E943E108091F00088608093F0004C
:102850000E94290EFF91EF91BF91AF919F918F91AF
:102860007F916F915F914F913F912F910F900FBE8C
:102870000F901F9018951F920F920FB60F92112470
:102880002F933F934F935F936F937F938F939F9378
:10289000AF93BF93CF93DF93EF93FF93C091E90082
:1028A000CF708091EC00D82FD17080FDD0E81092CD
:1028B000E9008091F000877F8093F00078940E9477
:1028C000C9111092E9008091F00088608093F000B7
:1028D000CD2BCF70C093E900FF91EF91DF91CF91A5
:1028E000BF91AF919F918F917F916F915F914F9128
:1028F0003F912F910F900FBE0F901F9018959093BE
:102900008502809384020895E0918402F09185020B
:10291000309721F00190F081E02D099480E0089536
:10292000EF92FF920F931F93CF93DF93E091840276
:10293000F09185023097B1F18C010280F381E02D96
:1029400009958091620382FF2DC080FF04C08BEA4D
:1029500094E00E94CA05E80118E085EAE82E84E0C8
:10296000F82E8091620380FF0BC088811F928F93A5
:10297000FF92EF920E9463060F900F900F900F90BE
:10298000115021961111EDCF8091620380FF0AC092
:1029900083EA94E0DF91CF911F910F91FF90EF9028
:1029A0000C94CA05DF91CF911F910F91FF90EF908A
:1029B0000895E0918402F0918502309721F004801F
:1029C000F581E02D09940895CF93DF932091820241
:1029D000309183022817390709F19093830280937D
:1029E0008202E0918402F09185023097B9F0EC0107
:1029F0000680F781E02D09958091620382FF0EC069
:102A000080FF0CC0DF93CF9385E994E09F938F9371
:102A10000E9463060F900F900F900F90DF91CF915F
:102A20000895CF93DF93209180023091810228177F
:102A3000390709F19093810280938002E09184022A
:102A4000F09185023097B9F0EC010084F185E02D1A
:102A500009958091620382FF0EC080FF0CC0DF9356
:102A6000CF9385E894E09F938F930E9463060F9025
:102A70000F900F900F90DF91CF9108950C94EE1569
:102A80000E9424220E945F0A0C94550BBF92CF92A1
:102A9000DF92EF92FF920F931F93CF93DF9300D0BB
:102AA00000D01F92CDB7DEB70E947A0907E812E086
:102AB000F12C8F2D0E94540AB82EF801C080C82630
:102AC00039F4F3940F5F1F4FF0E1FF12F2CF30C0E3
:102AD0008091620381FD0E940316D12CEE24E394C1
:102AE0008C2D8E21F9F0D982FA8291E08B2D8E21E6
:102AF00009F490E09B830E942D228160782F9D83B2
:102B00008C8349815A816B818D810E94391649815C
:102B10005A816B817C818D810E94A521F801808181
:102B20008E258083D394EE0CF8E0DF12D9CFC9CF85
:102B30008FEF89838A831B820E942D228160782FE8
:102B40009D838C8349815A816B818D810E943916C6
:102B50000E94A4210E94F6240E94B9060E948414B7
:102B600090918602891741F10E9484148093860215
:102B70009091620392FF0EC090FF0CC01F928F9342
:102B800086EB94E09F938F930E9463060F900F90C3
:102B90000F900F90809186020F900F900F900F90E2
:102BA0000F90DF91CF911F910F91FF90EF90DF90E9
:102BB000CF90BF900C94B6210F900F900F900F9074
:102BC0000F90DF91CF911F910F91FF90EF90DF90C9
:102BD000CF90BF9008950C945A0A08950895CF930A
:102BE000C62F0E94540A21E030E002C0220F331F9A
:102BF000CA95E2F790E02823392381E0232B09F4DA
:102C000080E0CF910895EF92FF920F931F93CF939F
:102C1000DF938FEC94E00E94CA05C0E0D0E083E32C
:102C2000E82E81E0F82E01EC14E08C2F0E94540A6B
:102C30000E949221FF92EF921F928F93DF93CF9386
:102C40001F930F930E94630621968DB79EB7089637
:102C50000FB6F8949EBF0FBE8DBFC031D10529F7C6
:102C6000DF91CF911F910F91FF90EF9008950895FC
:102C70000895CF93DF93CDB7DEB72B970FB6F894B7
:102C8000DEBF0FBECDBF942F4F83252F5887698796
:102C90007A878B874A855B85452B31F02F3F31F44E
:102CA00081E09F3F19F403C081E001C080E080FD16
:102CB00007C04F81588569857A858B850E94A5213B
:102CC000DE01119686E0FD0111928A95E9F785E013
:102CD000FE01379601900D928A95E1F749815A815C
:102CE0006B817C818D819E810E94FB1D2B960FB68E
:102CF000F894DEBF0FBECDBFDF91CF910895CF9383
:102D0000882309F4A9C0C82F8238A1F40E94841432
:102D100081FDA2C089E30E94EF200E9467212FEF6E
:102D200081EE94E0215080409040E1F700C0000027
:102D300089E315C08338C1F40E94841480FD8CC0DF
:102D400083E50E94EF200E9467212FEF81EE94E03F
:102D5000215080409040E1F700C0000083E50E94D0
:102D60000C21CF910C9467218438A1F40E94841423
:102D700082FD72C087E40E94EF200E9467212FEF3E
:102D800081EE94E0215080409040E1F700C00000C7
:102D900087E4E5CF8CEF8C0F813A20F080E58C0F33
:102DA0008E3248F48C2F0E942128811155C08C2F1F
:102DB0000E94EF20D6CF80E28C0F883048F4C77095
:102DC00081E001C0880FCA95EAF70E942D21C9CF82
:102DD0008BE58C0F833078F4C53A29F0C63A31F090
:102DE00083E890E005C081E890E002C082E890E0CE
:102DF000CF910C94E41488E58C0F853168F5C83ABE
:102E000089F0C93A91F0CA3A99F0CB3AA1F0CC3A9C
:102E1000A9F0CD3AB1F0CE3AB9F0CF3AC1F080E0A6
:102E200090E017C082EE90E014C089EE90E011C0EF
:102E30008AEE90E00EC085EB90E00BC086EB90E050
:102E400008C083EB90E005C084EB90E002C087EB04
:102E500090E0CF910C941115CF910895882309F437
:102E60006AC08238A1F40E94841481FF64C089E39F
:102E70000E94EF200E9467212FEF81EE94E0215005
:102E800080409040E1F700C0000089E315C083381E
:102E9000B9F40E94841480FF4EC083E50E94EF20A5
:102EA0000E9467212FEF81EE94E0215080409040F6
:102EB000E1F700C0000083E50E940C210C9467211B
:102EC0008438A1F40E94841482FF35C087E40E94F4
:102ED000EF200E9467212FEF81EE94E02150804087
:102EE0009040E1F700C0000087E4E6CF9CEF980F28
:102EF000913A10F390E5980F9E32F0F290E2980F1D
:102F0000983050F4877091E001C0990F8A95EAF7E4
:102F1000892F0E943321D2CF9BE5980F933020F464
:102F200080E090E00C94E414885A853120F480E02D
:102F300090E00C9411150895882321F00E942D2112
:102F40000C9467210895882321F00E9433210C946A
:102F5000672108950E944D210E941C210E94672133
:102F60000E949C250E94692480E090E00E94E41465
:102F700080E090E00C9411150E943D210C94AA175A
:102F8000CF92DF92EF92FF920F931F93CF93DF9335
:102F900000D000D01F92CDB7DEB76C010E94B821DF
:102FA000811101C385E0F601DE01119601900D92B9
:102FB0008A95E1F7F6014081518123813481211501
:102FC000310531F05F3F31F481E04F3F19F403C028
:102FD00081E001C080E080FDE6C2F601F280E5807C
:102FE000E2948FE0E82249835A83FB82722F3D836B
:102FF0002C836F2D8D810E9464208C010E946320A0
:103000000E94531FE12FE295EF708E2F90E0FC019C
:10301000EC5BFF4F0C94D22A812F807F1F70882396
:1030200011F01295107FFF2049F0112309F452C2CC
:10303000812F0E9440210E9467214CC2802F0E9454
:103040002E17112309F4AFC2812F0E9446210F9041
:103050000F900F900F900F90DF91CF911F910F91D4
:10306000FF90EF90DF90CF900C946721812F807FAD
:103070001F70803211F01295107F002319F001307B
:1030800009F12BC0FF20A9F0EE2059F1F1E0812FCA
:10309000EF1228C00F900F900F900F900F90DF91BC
:1030A000CF911F910F91FF90EF90DF90CF900C94F4
:1030B0005021EE2021F021E0E21609F474C20E94B2
:1030C00053212DC0FF20E9F085E08E1508F46BC276
:1030D0000E942A21812329F022C0FF20F1F0E11073
:1030E00015C0812F0F900F900F900F900F90DF91D0
:1030F000CF911F910F91FF90EF90DF90CF900C94A4
:103100009C1794E09E1508F44EC209C0F601858113
:1031100080FFE0C18F708583E4CFE110EEC1812F85
:1031200061C1812F86958695837019F08130B9F041
:103130003AC2FF2019F0C801937002C080E090E00D
:103140000F900F900F900F900F90DF91CF911F91E4
:103150000F91FF90EF90DF90CF900C94E414FF203C
:1031600019F0C801937002C080E090E00F900F90BA
:103170000F900F900F90DF91CF911F910F91FF90C3
:10318000EF90DF90CF900C941115802FFF2019F055
:103190000E947C2302C00E94E4230F900F900F90A6
:1031A0000F900F90DF91CF911F910F91FF90EF90B3
:1031B000DF90CF900C946924812F837009F070C048
:1031C000F110F1C1202F229526952770220F220F92
:1031D000602F6F70862F90E0A0E0B0E06C017D0161
:1031E000022E04C0CC0CDD1CEE1CFF1C0A94D2F78E
:1031F00004FF12C08FE090E0A0E0B0E004C0880FB0
:10320000991FAA1FBB1F2A95D2F7BC01CD0160955B
:1032100070958095909503C060E070E0CB011695A5
:10322000169513701230B1F040F56C297D298E2966
:103230009F29113031F10F900F900F900F900F9048
:10324000DF91CF911F910F91FF90EF90DF90CF9082
:103250000C94781F6C297D298E299F290F900F903F
:103260000F900F900F90DF91CF911F910F91FF90D2
:10327000EF90DF90CF900C94921F0E94781FC701AF
:10328000B6010F900F900F900F900F90DF91CF919C
:103290001F910F91FF90EF90DF90CF900C945E1FE5
:1032A000FF2019F0812F817001C08695882309F4D1
:1032B0007AC1202F229526952770220F220F602F8A
:1032C0006F70862F90E0A0E0B0E06C017D01022ECF
:1032D00004C0CC0CDD1CEE1CFF1C0A94D2F704FFCA
:1032E00012C08FE090E0A0E0B0E004C0880F991F0A
:1032F000AA1FBB1F2A95D2F7BC01CD01609570951E
:103300008095909503C060E070E0CB01169516950E
:1033100013701230B1F040F56C297D298E299F2958
:10332000113031F10F900F900F900F900F90DF91AF
:10333000CF911F910F91FF90EF90DF90CF900C9461
:103340003F206C297D298E299F290F900F900F9087
:103350000F900F90DF91CF911F910F91FF90EF9001
:10336000DF90CF900C9451200E943F20C701B601FE
:103370000F900F900F900F900F90DF91CF911F91B2
:103380000F91FF90EF90DF90CF900C942D20003F95
:10339000C1F128F480E4800F803250F096C0023FE3
:1033A00009F45EC008F449C0033F09F46CC08DC045
:1033B000F02FF071EF2E812F8F71FF2051F00E94BE
:1033C000C61F802FEE2019F08295807F8BCE8F70E4
:1033D00089CE0E94E71F802FEE2019F08295807F12
:1033E00001C08F700F900F900F900F900F90DF9192
:1033F000CF911F910F91FF90EF90DF90CF900C94A1
:10340000A317FF20A9F024E02E1508F4CCC0812FCB
:103410008F710F900F900F900F900F90DF91CF91C1
:103420001F910F91FF90EF90DF90CF900C940C20A4
:1034300085E08E1508F4B7C0EACFFF2099F0812F00
:103440008F710F900F900F900F900F90DF91CF9191
:103450001F910F91FF90EF90DF90CF900C94C61FBB
:10346000FF2069F3812F8F710F900F900F900F90B5
:103470000F90DF91CF911F910F91FF90EF90DF9010
:10348000CF900C94E71FFF2089F0812F8F710F9050
:103490000F900F900F900F90DF91CF911F910F9190
:1034A000FF90EF90DF90CF900C94B11F0F900F9092
:1034B0000F900F900F90DF91CF911F910F91FF9080
:1034C000EF90DF90CF900C94AC1FFF2099F0EE208E
:1034D00009F4B5CF802F0F900F900F900F900F90A1
:1034E000DF91CF911F910F91FF90EF90DF90CF90E0
:1034F0000C947F16EE2009F4B5CF802F0F900F901B
:103500000F900F900F90DF91CF911F910F91FF902F
:10351000EF90DF90CF900C942E17412F4F70602FBB
:10352000C6010E94F2220F900F900F900F900F9003
:10353000DF91CF911F910F91FF90EF90DF90CF908F
:103540000C94AE1E01112FC0FF2069F10E94BC1720
:103550009FEFE0E7F2E09150E040F040E1F700C07B
:1035600000000F900F900F900F900F90DF91CF9170
:103570001F910F91FF90EF90DF90CF900C949422C9
:10358000412F4F70602FC6010F900F900F900F903A
:103590000F90DF91CF911F910F91FF90EF90DF90EF
:1035A000CF900C94F5220F900F900F900F900F90EA
:1035B000DF91CF911F910F91FF90EF90DF90CF900F
:1035C00008951F93CF93DF9300D000D01F92CDB703
:1035D000DEB7942F4983252F5A836B837C838D8399
:1035E0004C815D81452B31F02F3F31F481E09F3FCD
:1035F00019F403C081E001C080E0182F117080FD34
:1036000031C049815A816B817C818D810E94642007
:10361000292F22952F702C3030F42A30A0F422501C
:10362000223030F022C02C30C9F02F30B9F01DC04C
:10363000853A28F48430C0F4823028F415C090E232
:10364000980F983088F0883E30F4803E68F48450BB
:10365000813A58F409C0803F41F406C093FB11271A
:1036600010F903C010E001C011E0812F0F900F90FE
:103670000F900F900F90DF91CF911F910895CF93EE
:10368000DF9300D000D01F92CDB7DEB70F900F9020
:103690000F900F900F90DF91CF910895CF93DF930C
:1036A00000D000D000D0CDB7DEB726960FB6F89484
:1036B000DEBF0FBECDBFDF91CF910895CF93DF93D3
:1036C000C091970280919802C817A1F0D0E0CE0176
:1036D00066E070E00E94AD2AFC01E756FD4F408194
:1036E000518162817381848195810E944E1B219654
:1036F000C770E8CFDF91CF9108954091C9025091F2
:10370000CA026091CB027091CC028091CD0290915F
:10371000CE020C944E1B1F93CF93DF938091CE0269
:1037200082958F7009F066C08091CB02882309F4DE
:1037300061C02091970210919802C091C902D09166
:10374000CA02E091CC02F091CD0281E0CF3F09F0B6
:1037500080E0482F211709F44DC0309721F0DF3F5A
:1037600021F080E003C081E001C0842F30E080FDC3
:103770003DC0C90166E070E00E94AD2ADC01A75699
:10378000BD4F11968C9111978D1330C08C918C1375
:103790002DC012968C911297811128C013968D918D
:1037A0009C9114978E179F0708F401978E1B9F0B0F
:1037B000883C9105D8F48091CE028F70806180930F
:1037C000CE02C90166E070E00E94AD2AFC01E2561B
:1037D000FD4F90819F709061908389EC92E00E94F0
:1037E000C017DF91CF911F910C945E1B2F5F3F4F4D
:1037F0002770B0CFDF91CF911F910895AF92BF9204
:10380000CF92DF92EF92FF920F931F93CF93DF93AC
:10381000CDB7DEB761970FB6F894DEBF0FBECDBF50
:103820007C0185E0F701DE011D9601900D928A95DD
:10383000E1F7D7014C9111962C9111971296DC90DB
:10384000129713960D911C9114975091C902609193
:10385000CA028091CC029091CD02009731F06F3F67
:1038600031F431E05F3F19F403C031E001C030E0D2
:10387000B32FB170BB2E30FD76C1A090CB02AA2031
:1038800009F4D2C03091CE020817190728F0F801C8
:10389000E81BF90BCF0104C080959095800F911F14
:1038A000CC24C394883C910588F0C12C307F09F06A
:1038B000A6C0702F198B088B522F6D2D89890E94FD
:1038C0003F1B89EC92E00E94C017C3C0832F807F0A
:1038D00009F059C0261315C0451313C0CD2CD110C3
:1038E00010C03F7030613093CE020E947D1B89EC86
:1038F00092E00E94C0178091CE02D70115968C935A
:1039000068C10115110531F02F3F31F481E04F3FBF
:1039100019F403C081E001C080E080FD03C081E0B4
:103920008D2502C080E090E0B82FB170CB2E80FFD3
:103930001FC0E091970230919802E31709F425C166
:10394000F0E0CF0166E070E00E94AD2ADC01A756EE
:10395000BD4F11968C911197281307C08C91481375
:1039600004C012968C91D81203C03196E770E5CF4F
:10397000CD2CDD2009F42DC18091CE028160809391
:10398000CE02C12C26C1261308C0451306C0D11093
:1039900004C08091CE02D701B9C04D872E87DF8643
:1039A000702F198B088B522F6D2D89890E94E11A77
:1039B0008823A1F1DD2091F12091CE02822F829502
:1039C0008F7090E0029774F08091C9029091CA02C2
:1039D00098878F8319861B870A872C87CE010796C5
:1039E0000E94C01786E0F701A9ECB2E001900D92A9
:1039F0008A95E1F70E948B1B0E947D1B12C026173F
:103A000091F14D872E87DF86702F198B088B522FEF
:103A10006D2D89890E94E11A811139C0C7010E9468
:103A2000C017CC24C394D5C00817190708F447C0A1
:103A3000F801E81BF90BCF01883C910508F444C05C
:103A4000C12C702F198B088B522F6D2D89890E94E4
:103A50003F1BE9ECF2E086E0DF011D928A95E9F771
:103A60000E947D1BB6C04513CCCFD110CACF809128
:103A7000CE02F7018583C7010E94C01786E0E9ECFA
:103A8000F2E0DF011D928A95E9F7CA2CA2C0DD2081
:103A900029F22091CE02822F82958F7090E00297BA
:103AA0000CF4A0CF8091C9029091CA029A838983B5
:103AB0001B821D830C832E83CE01019691CF8095AE
:103AC0009095800F911FB8CFCD2CDD2009F4A6CFA3
:103AD000261333C0451331C02091CE0220FD24C0EF
:103AE000822F82958F70482F50E041155105E1F0EB
:103AF000D70115962C9315974F30510549F08F5FDC
:103B0000982F9295907F822F8F70892B15968C938A
:103B1000C7010E94C01786E0F701A9ECB2E001904E
:103B20000D928A95E1F79CCF86E0F701A9ECB2E00F
:103B300001900D928A95E1F74CC04D872E87DF8664
:103B4000702F198B088B522F6D2D89890E94E11AD5
:103B5000811148CF8091CE0281608093CE02C7014F
:103B60000E94C01736C0DD2009F458CF4D872E873C
:103B7000DF86702F198B088B522F6D2D89890E943B
:103B8000E11A882309F44ACF2DCF702F198B088BA7
:103B9000522F6D2D89890E946420292F22952F7024
:103BA000223028F49F7039F0811105C00BC02430F9
:103BB00028F49F7049F4805E883020F0C7010E948D
:103BC000C017BC2CCB2C05C0F7019581907F99F7CD
:103BD000F9CF8C2D61960FB6F894DEBF0FBECDBF26
:103BE000DF91CF911F910F91FF90EF90DF90CF90D9
:103BF000BF90AF900895CF93DF93CDB7DEB72C97EA
:103C00000FB6F894DEBF0FBECDBF4F8358876987CC
:103C10007A878B879C87CE0107960E94FE1B88239C
:103C2000D1F09F8188852A853B85232B31F08F3FFA
:103C300031F481E09F3F19F403C081E001C080E0CE
:103C400080FD6FC04F81588569857A858B859C85FD
:103C50000E944E1B66C086E0FE013796DE0111967B
:103C600001900D928A95E1F7FF81E8856A857B8551
:103C70006115710531F0EF3F31F481E0FF3F19F438
:103C800003C081E001C080E080FD4BC080919802BC
:103C900090E09C012F5F3F4F2770332740919702A0
:103CA00050E02417350709F443C0F983EA837D8384
:103CB0006C8366E070E00E94AD2ADC01A756BD4F20
:103CC00096E0FE01319601900D929A95E1F72093CE
:103CD00098020E945E1B25C090E066E070E00E94A2
:103CE000AD2A87569D4F0E94FE1B882371F180915B
:103CF000970290E066E070E00E94AD2AFC01E75672
:103D0000FD4F4081518162817381848195810E9440
:103D10004E1B8091970290E00196877099278093BF
:103D2000970280919702909198028913D5CF0DC088
:103D30000E94BC171092980210929702E9ECF2E0F0
:103D400086E0DF011D928A95E9F72C960FB6F8946C
:103D5000DEBF0FBECDBFDF91CF910895DF92EF920E
:103D6000FF920F931F93CF93DF93FC01892B09F4EC
:103D700088C0E12CF12CDD24D394EF0121968491AD
:103D8000853709F460C058F4843708F04EC0843099
:103D900008F068C08130D1F0823071F172C088378C
:103DA00009F45BC050F4863709F453C0873709F033
:103DB00068C08E2D0E943A2152C09CE7980F903720
:103DC00008F05FC08F770E942E174EC08F010E5FE4
:103DD0001F4FFE01849190E2980F983050F4877045
:103DE000FD2D01C0FF0F8A95EAF78F2F0E94402119
:103DF00015C00E947F1614C08F010E5F1F4FFE0179
:103E0000849190E2980F983068F48770FD2D01C07E
:103E1000FF0F8A95EAF78F2F0E9446210E946721A3
:103E2000E80122C00E942E17FBCFCF010296FE01AF
:103E3000C491CC2361F0EFE9FFE03197F1F700C0C6
:103E40000000C150F6CFCF010296FE01F490EC01C4
:103E50000BC00E942A21E82E07C00E943D210E942B
:103E6000672102C00E947F168F2D882341F0EFE961
:103E7000FFE03197F1F700C000008150F6CFFE015E
:103E80007CCFDF91CF911F910F91FF90EF90DF904A
:103E9000089560934F037093500380935103909360
:103EA00052030C94B5210895609353037093540307
:103EB00080935503909356030C94B4210F931F9352
:103EC00000915303109154032091550330915603F0
:103ED000602B712B822B932B6093530370935403AD
:103EE00080935503909356031F910F910C94B42126
:103EF0000F931F9300915303109154032091550386
:103F000030915603602371238223932360935303DC
:103F10007093540380935503909356031F910F9110
:103F20000C94B4210F931F930091530310915403E9
:103F300020915503309156036027712782279327DC
:103F400060935303709354038093550390935603E7
:103F50001F910F910C94B42160E070E0CB010C94A0
:103F6000491F0F931F9341E050E060E070E08A0129
:103F70009B0104C0000F111F221F331F8A95D2F727
:103F8000C901B8011F910F910C94491F0F931F9302
:103F900041E050E060E070E004C0440F551F661F30
:103FA000771F8A95D2F780914F0390915003A0918B
:103FB0005103B09152038A019B01082B192B2A2B24
:103FC0003B2BC901B8011F910F910C94491F0F930E
:103FD0001F9341E050E060E070E004C0440F551FC3
:103FE000661F771F8A95D2F740955095609570951A
:103FF00080914F0390915003A0915103B0915203CF
:104000008A019B01082319232A233B23C901B801F4
:104010001F910F910C94491F0F931F9341E050E0A3
:1040200060E070E004C0440F551F661F771F8A953B
:10403000D2F780914F0390915003A0915103B0911A
:1040400052038A019B01082719272A273B27C90108
:10405000B8011F910F910C94491F0F931F9300916A
:104060004F03109150032091510330915203602B64
:10407000712B822B932B1F910F910C94491F0F933F
:104080001F9300914F0310915003209151033091E1
:10409000520360237123822393231F910F910C9469
:1040A000491F0F931F9300914F03109150032091CC
:1040B00051033091520360277127822793271F9164
:1040C0000F910C94491F08958F929F92AF92BF92C7
:1040D000DF92EF92FF920F931F93CF93DF9300D065
:1040E00000D01F92CDB7DEB76B837C838D838A01AE
:1040F0008C819D81892B31F01F3F31F481E04F3F4E
:1041000019F403C081E001C080E080FF03C080E0BB
:1041100090E054C08B81882309F43DC080904F0308
:1041200090905003A0905103B0905203809153039C
:1041300090915403A0915503B0915603882A992A6F
:10414000AA2ABB2A2FE1E22EF12CD501C4010E2CA4
:1041500004C0B695A795979587950A94D2F780FDE8
:1041600006C081E0E81AF10880F7D12C07C0DE2CE8
:10417000B8018E2D0E94C522019799F3E12FF0E03E
:1041800093E0EE0FFF1F9A95E1F7E153FD4FE00F2B
:10419000F11DD0820CC0E12FF0E083E0EE0FFF1F95
:1041A0008A95E1F7E153FD4FE00FF11DD0800983BF
:1041B0001A8369817A818D2D0E94C5220F900F90FC
:1041C0000F900F900F90DF91CF911F910F91FF9063
:1041D000EF90DF90BF90AF909F908F9008952091C7
:1041E000250130912601F90132969FEF40E051916F
:1041F000851789F09F3F19F4511101C0942F4F5F2B
:104200004630A9F79F3F39F0F901E90FF11D97FDFD
:10421000FA95828308950895E0912501F091260191
:104220009F012A5F3F4F9281891301C0128231960C
:10423000E217F307C1F7089581E090E0E0912501CE
:10424000F0912601E80FF91F108201968830910540
:10425000A9F7089580916103089590916103892BD6
:1042600080936103089580959091610389238093E1
:104270006103089580936103089510926103089586
:1042800090916003892B80936003089580959091AD
:10429000600389238093600308951092600308955A
:1042A0008093570308951092570308958091250134
:1042B00090912601FC0131969C01285F3F4F80E0E0
:1042C000919191118F5FE217F307D1F70895E09173
:1042D0002501F0912601809161038083E091250101
:1042E000F0912601908180916003892B80838091D9
:1042F0005703882361F0E0912501F0912601908118
:10430000892B80830E94562181111092570380913E
:104310002501909126010C94901490935301809361
:10432000520108958295982F9373292F220F220FFF
:10433000982F9C7C96959695922B892F8575880F42
:104340009A7A9695892B08950895CF93DF9300D09C
:1043500000D01F92CDB7DEB70F900F900F900F9047
:104360000F90DF91CF910895089508950C94EB1567
:1043700080E0089580917703843021F110926303E7
:1043800020E488E190E00FB6F894A895809360004F
:104390000FBE2093600083B7817F846083BF83B7A3
:1043A000816083BF7894889583B78E7F83BF0FB673
:1043B000F894A895809160008861809360001092C5
:1043C00060000FBE0895CF930E9437160E947A09AD
:1043D0000E943816C0E08C2F0E94540A811104C03C
:1043E000CF5FC031C1F701C081E0CF9108950E9435
:1043F000ED150C94BC171F920F920FB60F9211245B
:104400008F939F93AF93BF9380916303811113C0E8
:104410008091640390916503A0916603B091670356
:104420004196A11DB11D8093640390936503A093F1
:104430006603B0936703BF91AF919F918F910F90E7
:104440000FBE0F901F90189582E084BD93E095BD3C
:104450009AEF97BD80936E0008952FB7F8948091DE
:10446000640390916503A0916603B09167032FBF29
:1044700008952FB7F894609164037091650380915B
:104480006603909167032FBF0895CF92DF92EF925A
:10449000FF920F931F932FB7F894409164035091AC
:1044A000650360916603709167032FBF6A017B010A
:1044B000EE24FF248C0120E030E0C016D106E20695
:1044C000F30610F4415051099A01281B390BC90118
:1044D0001F910F91FF90EF90DF90CF9008951F9262
:1044E0000F920FB60F9211248F939F93AF93BF93A8
:1044F0008091640390916503A0916603B091670376
:104500000196A11DB11D8093640390936503A09350
:104510006603B0936703BF91AF919F918F910F9006
:104520000FBE0F901F9018950E942913F89487E7EB
:1045300097E7909301088093000887E090EBDC01F7
:104540008093800390938103A0938203B0938303AD
:104550009CE088E10FB6F894A895809360000FBEA8
:1045600090936000FFCFE92FF0E093E0EE0FFF1F84
:104570009A95E1F7E80FF11DE855FF4F8491982FC8
:1045800092959F708F7097700895CF93C82FCB012D
:104590000E94B322292F30E054E0220F331F5A9596
:1045A000E1F7282B203831051CF080E090E018C09E
:1045B000EC2FF0E023E0EE0FFF1F2A95E1F7977054
:1045C000E90FF11D34E0EE0FFF1F3A95E1F78F7010
:1045D000E80FF11DEE0FFF1FE050F849859194910F
:1045E000CF91089580E090E00895089580916A0346
:1045F00080FF0CC080912A0190E065E070E00E948D
:10460000AD2A95958795959587952EC081FF0AC00F
:1046100080912A0190E065E070E00E94AD2A9595B6
:10462000879522C082FF08C080912A0190E065E052
:1046300070E00E94AD2A18C020916B032223D9F0AC
:1046400030912901231780F780912A0190E065E0DD
:1046500070E00E94AD2A622F70E00E94AD2A632FA5
:1046600070E00E94BE2ACB018038910538F4009793
:1046700039F481E005C085E090E008958FE7089562
:10468000089580916A0380FF08C06091280170E05E
:10469000759567957595679523C081FF06C06091F4
:1046A000280170E0759567951BC082FF04C060917A
:1046B000280170E012C060916B036623A9F020917D
:1046C00027016217A0F78091280170E090E00E9416
:1046D000AD2A622F70E00E94BE2A6038710540F456
:1046E0006115710519F406C061E070E0862F089528
:1046F0008FE7089581E00895803F21F40E94F6221B
:10470000819504C0813F29F40E94F62280936E03B4
:104710000895823F21F40E94F622819504C0833FD0
:1047200029F40E94F62280936D030895893F19F4BD
:104730000E94412305C08A3F31F40E9441238195A4
:1047400080936F0308958B3F21F40E94412381954C
:1047500004C08C3F29F40E94412380937003089584
:10476000843F21F480916C03816017C0853F21F460
:1047700080916C03826011C0863F21F480916C03AC
:1047800084600BC0873F21F480916C03886005C072
:10479000883F31F480916C03806180936C030895AD
:1047A0008D3F21F480916A0381600BC08E3F21F41C
:1047B00080916A03826005C08F3F29F480916A036B
:1047C000846080936A030895803F39F480916E037A
:1047D00087FF6CC010926E0369C0813F29F48091FD
:1047E0006E031816BCF362C090916D03823F29F4EA
:1047F00097FF5CC010926D0359C0833F19F41916DE
:10480000CCF354C0893F41F480916F0318160CF02B
:104810004DC010926F034AC08A3F29F480916F0304
:1048200087FF44C0F6CF8B3F39F48091700387FF38
:104830003DC0109270033AC08C3F29F48091700300
:104840001816BCF333C0843F21F480916C038E7F33
:1048500017C0853F21F480916C038D7F11C0863F86
:1048600021F480916C038B7F0BC0873F21F48091F2
:104870006C03877F05C0883F31F480916C038F7E85
:1048800080936C0313C08D3F21F480916A038E7F67
:104890000BC08E3F21F480916A038D7F05C08F3F4E
:1048A00029F480916A038B7F80936A0380916D0362
:1048B00081110EC080916E0381110AC080916F0337
:1048C000811106C080917003811102C010926B03A8
:1048D00008958091620383FF7EC084E095E00E948A
:1048E000CA0580916C031F928F938FEF94E09F9382
:1048F0008F930E9463068DEF94E00E94CA05809119
:104900006D03282F082E000C330B3F938F938AEFF3
:1049100094E09F938F930E94630688EF94E00E9437
:10492000CA0580916E03282F082E000C330B3F938D
:104930008F9385EF94E09F938F930E94630683EF9C
:1049400094E00E94CA0580916F03282F082E000C66
:10495000330B3F938F9380EF94E09F938F930E944C
:1049600063068EEE94E00E94CA0580917003282FA2
:10497000082E000C330B3F938F938BEE94E09F93A4
:104980008F930E94630688EE94E00E94CA0580918E
:104990006B031F928F9385EE94E09F938F930E94F9
:1049A000630683EE94E00E94CA0580916A031F9219
:1049B0008F9380EE94E09F938F930E9463068DED1A
:1049C00094E00E94CA058DB79EB74C960FB6F89436
:1049D0009EBF0FBE8DBF8CE693E00E94D9140E944B
:1049E0002D22909369038093680308951F93CF93BA
:1049F000DF9380916803909169030E944522FC0136
:104A000020916B03222321F080912B0190E007C0BD
:104A100080912C0190E06AE070E00E94AD2AE817D6
:104A2000F90708F485C080916D03C0916E03D091A1
:104A30006F0310917003811107C0C11175C0D111AE
:104A400073C0111171C074C02F3F19F02F5F2093F4
:104A50006B03181624F40E94F62280936D03809154
:104A60006D0387FF05C00E94F622819580936D0338
:104A70001C1624F40E94F62280936E0380916E032C
:104A800087FF05C00E94F622819580936E03609196
:104A90006D03662331F1C0916E03CC2311F1062E14
:104AA000000C770B880B990B0E94AC2923E333E3AE
:104AB00043E35FE30E94102A0E94742960936D0310
:104AC0006C2FCC0F770B880B990B0E94AC2923E33A
:104AD00033E343E35FE30E94102A0E94742960934A
:104AE0006E031D1624F40E94412380936F0380916E
:104AF0006F0387FF05C00E944123819580936F0358
:104B0000111624F40E944123809370038091700356
:104B100087FF05C00E944123819580937003DF9138
:104B2000CF911F910C9469242F3F09F08FCFA0CF14
:104B3000DF91CF911F910895ECE6F3E085E0DF016E
:104B40001D928A95E9F710926B0310926A030895FB
:104B500087E297E00E94CA051F9281E08F931F921F
:104B600085E08F9389ED96E09F938F930E94630673
:104B70000F900F900F900F900F900F90089583302B
:104B8000E9F128F4813061F0823009F1089585302F
:104B900009F462C008F449C0863009F474C008956D
:104BA00080912C01262F30E0280F311D2F3F310539
:104BB00024F4680F60932C0103C08FEF80932C01C5
:104BC00080912C011F928F9382E196E072C08091B8
:104BD0002B01262F30E0280F311D2F3F310524F403
:104BE000680F60932B0103C08FEF80932B0180919E
:104BF0002B011F928F9380E096E05BC080912A0189
:104C0000262F30E0280F311D2F3F310524F4680F87
:104C100060932A0103C08FEF80932A0180912A01BB
:104C20001F928F938DEE95E044C080912901262F2D
:104C300030E0280F311D2F3F310524F4680F6093B9
:104C4000290103C08FEF80932901809129011F92D0
:104C50008F9388ED95E02DC080912801262F30E0BC
:104C6000280F311D2F3F310524F4680F6093280170
:104C700003C08FEF80932801809128011F928F93AA
:104C80008FEB95E016C080912701262F30E0280F8A
:104C9000311D2F3F310524F4680F6093270103C0B5
:104CA0008FEF80932701809127011F928F9384EAD1
:104CB00095E09F938F930E9463060F900F900F9043
:104CC0000F900895833081F128F4813059F08230BB
:104CD000D1F00895853009F449C0B8F1863009F45F
:104CE00056C0089580912C01681720F4861B80938C
:104CF0002C0102C010922C0180912C011F928F93E5
:104D000085E995E054C080912B01681720F4861B3B
:104D100080932B0102C010922B0180912B011F92D6
:104D20008F9383E895E043C080912A01681720F4AF
:104D3000861B80932A0102C010922A0180912A01C9
:104D40001F928F9380E795E032C080912901681708
:104D500020F4861B8093290102C0109229018091C2
:104D600029011F928F938BE595E021C08091280146
:104D7000681720F4861B8093280102C01092280136
:104D8000809128011F928F9382E495E010C080915A
:104D90002701681720F4861B8093270102C0109218
:104DA0002701809127011F928F9387E295E09F93BF
:104DB0008F930E9463060F900F900F900F900895AD
:104DC000CF93C82F1F928F938CE298E09F938F937D
:104DD0000E94630681E090E0A0E0B0E0BC01CD015C
:104DE00004C0660F771F881F991FCA95D2F70E94CB
:104DF000541F0F900F900F900F90CF910C94BC17F1
:104E0000CF93873288F58E3108F00BC18E3009F4CC
:104E100087C0D8F4873009F460C08B3009F44FC0E4
:104E2000863009F002C180916203817F8E7F80937A
:104E3000620381E398E00E94CA0583EE9AE00E9433
:104E4000CA0581E08093720346C0863109F4B0C080
:104E500020F4803109F47AC0E8C0893109F491C0A6
:104E60008B3109F449C0E1C0883349F150F48932EB
:104E700009F4D5C0853309F4D2C0873209F0D5C012
:104E8000CEC0833409F4CBC028F48A3308F4CDC0F3
:104E90008953C8C0883409F0C8C00E94BC1782ED8D
:104EA0009AE00E94CA052FEF83ED90E321508040E5
:104EB0009040E1F700C000000E9494220CC088E5F9
:104EC00098E041C089EB9AE00E94CA058091620394
:104ED000816080936203C1E0ADC080916203C82FFE
:104EE000C17080FFEFCF85EC9AE00E94CA058091E7
:104EF0006203817F8E7F3FC09091620391FBCC273C
:104F0000C0F981E0C827892FC0FB81F98093620333
:104F1000CC2319F08CEA9AE029C08EE99AE013C0FC
:104F20009091620392FBCC27C0F981E0C827892FBA
:104F3000C0FB82F980936203CC2319F08FE89AE0DA
:104F400015C08FE79AE00E94CA05C5CF9091620311
:104F500093FBCC27C0F981E0C827892FC0FB83F9D8
:104F600080936203CC2351F083E79AE00E94CA0544
:104F7000809162038160809362035CC086E69AE060
:104F8000E2CF87E59AE00E94CA0584E39AE00E9496
:104F9000CA058FEE99E00E94CA0587EC99E00E944D
:104FA000CA0582E899E00E94CA0586E599E0CBCF60
:104FB00088E499E00E94CA050E9484141F928F938E
:104FC0008EE299E09F938F930E9463068091240163
:104FD0001F928F9387E199E09F938F930E946306BE
:104FE00080917F021F928F9384E099E09F938F932B
:104FF0000E9463060E9439229F938F937F936F9341
:105000008DEE98E09F938F930E9463068DB79EB7B5
:1050100042960FB6F8949EBF0FBE8DBF5CCF80E066
:1050200001C08D510E94E02656CF8BEE98E00E9481
:10503000CA05C0E08C2FCF91089580E008950C94AC
:105040001D28CF93C82F80917203813069F020F022
:10505000823009F449C040C167E08FE00E94EF153B
:10506000882309F43FC106C067E08FE00E94EF1576
:10507000882361F08C2F0E941F28811104C08C2F7F
:105080000E9400272FC081E090E02CC08C2F0E944E
:105090001D28811126C0C431E1F070F4CB3081F0BD
:1050A000C031D1F40E94A82584E298E00E94CA058C
:1050B00082E08093720315C0C93259F0C83361F49D
:1050C00081E398E00E94CA0588E298E00E94CA0540
:1050D00008C01092720304C182E298E00E94CA05DF
:1050E000FFC081E08170FEC0C43228F5CE3108F0E7
:1050F000C1C0CB30A1F1D0F4C73009F0D3C08EE1EC
:1051000080932C0182E380932B018AE080932A0113
:1051100084E18093290188E08093280188E28093CC
:10512000270188EC96E00E94CA05BFC0C33149F14F
:10513000C431C1F0B7C0CB3409F4A9C028F4C932D6
:1051400089F0C83361F0AEC0C13509F49EC0C235E4
:1051500009F499C0CE3409F0A5C06AE09EC00E944F
:10516000A825A3C080917103882319F010927103C0
:105170009CC085ED96E00E94CA0581E08093720391
:10518000B1C08FEA96E00E94CA058DE996E00E94C0
:10519000CA0580912C011F928F938AE996E09F9314
:1051A0008F930E94630688E996E00E94CA0586E80C
:1051B00096E00E94CA0580912B011F928F9383E88D
:1051C00096E09F938F930E94630681E896E00E9489
:1051D000CA0582E796E00E94CA0580912A011F92C3
:1051E0008F938FE696E09F938F930E9463068DE6E0
:1051F00096E00E94CA058CE596E00E94CA0580915F
:1052000029011F928F9389E596E09F938F930E94C7
:10521000630687E596E00E94CA0582E496E00E9454
:10522000CA05809128011F928F938FE396E09F9388
:105230008F930E9463068DE396E00E94CA0586E282
:1052400096E00E94CA05809127011F928F9383E206
:1052500096E09F938F930E94630681E296E00E94FE
:10526000CA058DB79EB748960FB6F8949EBF0FBE7D
:105270008DBF1BC0CE51EC2FF0E0E85BFE4F80816C
:105280008093710312C061E003C061E006C06AE070
:10529000809171030E94BF2508C0809171030E9414
:1052A000622603C086EC96E013C0809171038823C8
:1052B00069F01F928F9380EC96E09F938F930E94EA
:1052C00063060F900F900F900F9004C08DEB96E047
:1052D0000E94CA0581E006C01092720380E002C0FD
:1052E00080E000CFCF9108950E947B296894B1118E
:1052F0000C940A2A08950E94EF2988F09F5798F08D
:10530000B92F9927B751B0F0E1F0660F771F881FCA
:10531000991F1AF0BA95C9F714C0B13091F00E94E4
:10532000092AB1E008950C94092A672F782F88275D
:10533000B85F39F0B93FCCF3869577956795B3950B
:10534000D9F73EF490958095709561957F4F8F4F7A
:105350009F4F0895E89409C097FB3EF4909580957F
:10536000709561957F4F8F4F9F4F9923A9F0F92F2B
:1053700096E9BB279395F695879577956795B795A9
:10538000F111F8CFFAF4BB0F11F460FF1BC06F5F8F
:105390007F4F8F4F9F4F16C0882311F096E911C0A1
:1053A000772321F09EE8872F762F05C0662371F0C2
:1053B00096E8862F70E060E02AF09A95660F771FD6
:1053C000881FDAF7880F9695879597F9089557FD06
:1053D0009058440F551F59F05F3F71F04795880F63
:1053E00097FB991F61F09F3F79F0879508951216FA
:1053F00013061406551FF2CF4695F1DF08C01616A6
:1054000017061806991FF1CF869571056105089456
:105410000895E894BB2766277727CB0197F908956D
:105420000E94222A0C949C2A0E948E2A38F00E9404
:10543000952A20F0952311F00C94852A0C948B2A40
:105440000C940A2A0E94E72978F39923C9F355237B
:10545000B9F3950F50E0551FAA27EE27FF27BB276A
:1054600000240894679520F4E20FF31FB41F0A1E6E
:10547000220F331F441FAA1F6695A9F7779530F4B2
:10548000F30FB41F0A1E121E08F46395330F441F56
:10549000AA1F221F769599F7879520F4B40F0A1E4C
:1054A000121E631F440FAA1F221F331F8695A9F7E0
:1054B000862F712D602D11249F5750409AF0F1F0E6
:1054C00088234AF0EE0FFF1FBB1F661F771F881F40
:1054D00091505040A9F79E3F510580F00C94852AC9
:1054E0000C940A2A5F3FE4F3983ED4F386957795AF
:1054F0006795B795F795E7959F5FC1F7FE2B880FE6
:10550000911D9695879597F9089597F99F6780E87B
:1055100070E060E008959FEF80EC089500240A9405
:105520001616170618060906089500240A9412167E
:105530001306140605060895092E0394000C11F4B1
:10554000882352F0BB0F40F4BF2B11F460FF04C05E
:105550006F5F7F4F8F4F9F4F08950024552704C0E2
:10556000080E591F880F991F009729F076956795A7
:10557000B8F37105B9F7802D952F089597FB072E85
:1055800016F4009407D077FD09D00E94D82A07FCB2
:1055900005D03EF4909581959F4F08957095619543
:1055A0007F4F0895EE0FFF1F0590F491E02D0994B1
:1055B000AA1BBB1B51E107C0AA1FBB1FA617B70739
:1055C00010F0A61BB70B881F991F5A95A9F7809555
:0C55D0009095BC01CD010895F894FFCF28
:1055DC00FFFFA514000069FFFF27E78C000000FF08
:1055EC00FF9464000576010000FF640CF40CD10CF0
:1055FC009B0C670C0158032808140A321E7965733A
:10560C00006E6F00404D36224504F803C203A00320
:10561C002C0345035E037703010203040506070808
:02562C00090073
:106800008800EA44E944E244040005000600070069
:10681000080009000A000B000C000D000E000F001C
:1068200010001100120013001400150016001700CC
:10683000180019001A001B001C001D001E001F007C
:10684000200021002200230024002500260027002C
:10685000280029002A002B002C002D002E002F00DC
:10686000300031A232003300340035A13600370049
:10687000380082003A003B003C003D003E003F00F3
:1068800040004100420043004400450046004700EC
:10689000480049004A004B004C004D004E004F009C
:1068A000500051005200530067005400550056003C
:1068B000580059005A005B005C005D005E005F00FC
:1068C00060006100620063006400650057006700BB
:1068D000CD4469006A006B006C006D006E006F00B3
:1068E0007000710072006620890087008A008B00AA
:1068F000E000E100E200E300E400E500E600E7007C
:106900008800010001000100EA4401000100E244A6
:106910000100010001000100460001004A004B0097
:10692000010001004700480001000100E9440100A6
:106930000100010001000100010001003A003B00DC
:106940003C003D003E003F0040004100420043004B
:10695000010035004C0001000100440045005200D8
:1069600049000100010050004F0029004D004E0079
:1069700051000100010001000100010001000100BF
:1069800001000100010001000100010001000100FF
:1069900001000100010001000100010001004D00A3
:1069A0004A004E004B0001000100010001000100FF
:1069B00001000100010001000100010001000100CF
:1069C00001000100010001000100650001006700F5
:1069D000010069006A006B006C006D006E006F00C2
:1069E0007000710072000100890087008A008B002E
:1069F0000100010001000100010001000100E700A9
:106A00008800010001000100EA4401000100E244A5
:106A10000100010001000100460001004A004B0096
:106A2000010001004700480001000100E9440100A5
:106A30000100010001000100010001003A003B00DB
:106A40003C003D003E003F0040004100420043004A
:106A5000010035004C0001000100440045005200D7
:106A600049000100010050004F0029004D004E0078
:106A700051000100010001000100010001000100BE
:106A800001000100010001000100010001000100FE
:106A900001000100010001000100010001004D00A2
:106AA0004A004E004B0001000100010001000100FE
:106AB00001000100010001000100010001000100CE
:106AC00001000100010001000100650001006700F4
:106AD000010069006A006B006C006D006E006F00C1
:106AE0007000710072000100890087008A008B002D
:106AF0000100010001000100010001000100E700A8
:00000001FF
